:1000000012C0189518951895189518951895189563
:100010001895189518951895189518951895189578
:100020001895189518958FED8DBFC0ECE8EB4E2E06
:10003000DD275D2EEEE7F0E0A0E6B0E088278D93A7
:100040003197E9F7E8D2662488EF8ABB8FE087BB57
:100050008BEE81BB87E08BBB8FE788BB84E182BBE3
:100060008CE021D3BED2E4E7F7E0B3D2B8D2E4E823
:10007000F7E0AFD2E3E0F0E0C5D2BF98A7E69C91ED
:1000800097FF04C0B7990EC09F779C93B79B0AC097
:1000900088E29F93992733D39F91B79B03C09068C1
:1000A0009C934FD2E9E0F0E0A6E691E05CD30091AA
:1000B00066000E3C08F004C085B7806385BF889554
:1000C00080E080936400A1E62DD380E080936300FC
:1000D00080E08093650085D2EEE8F7E07AD28FE782
:1000E00088BBC09AC39881E080936000BE98A7E661
:1000F0009C9196FF04C0B69B0EC09F7B9C93B699C3
:100100000AC088E29F939927FAD29F91B69903C0BB
:1001100090649C9313D182E080936000BD98A7E621
:100120009C9195FF04C0B59B0EC09F7D9C93B59993
:100130000AC088E29F939927E2D29F91B59903C0A4
:1001400090629C93FBD083E080936000BC98A7E60C
:100150009C9194FF04C0B49B0EC09F7E9C93B49965
:100160000AC088E29F939927CAD29F91B49903C08D
:1001700090619C93E3D0C39AC29884E0809360001E
:10018000BE98A7E69C9196FF04C0B69B0EC09F7BCD
:100190009C93B6990AC088E29F939927B0D29F9109
:1001A000B69903C090649C93C9D085E080936000A9
:1001B000BD98A7E69C9195FF04C0B59B0EC09F7D9E
:1001C0009C93B5990AC088E29F93992798D29F91F2
:1001D000B59903C090629C93B1D086E08093600093
:1001E000BC98A7E69C9194FF04C0B49B0EC09F7E70
:1001F0009C93B4990AC088E29F93992780D29F91DB
:10020000B49903C090619C9399D0C29AC19887E039
:1002100080936000BE98A7E69C9196FF04C0B69BB1
:100220000EC09F7B9C93B6990AC088E29F93992742
:1002300066D29F91B69903C090649C937FD088E06A
:1002400080936000BD98A7E69C9195FF04C0B59B84
:100250000EC09F7D9C93B5990AC088E29F93992711
:100260004ED29F91B59903C090629C9367D089E06C
:1002700080936000BC98A7E69C9194FF04C0B49B57
:100280000EC09F7E9C93B4990AC088E29F939927E1
:1002900036D29F91B49903C090619C934FD0C19A7C
:1002A000C0988BE080936000BE98A7E69C9196FF73
:1002B00004C0B69B0EC09F7B9C93B6990AC088E28F
:1002C0009F9399271CD29F91B69903C090649C93E9
:1002D00035D08AE080936000BD98A7E69C9195FF99
:1002E00004C0B59B0EC09F7D9C93B5990AC088E25F
:1002F0009F93992704D29F91B59903C090629C93D4
:100300001DD08CE080936000BC98A7E69C9194FF80
:1003100004C0B49B0EC09F7E9C93B4990AC088E22F
:100320009F939927ECD19F91B49903C090619C93BE
:1003300005D08AE090E0E3D1D4CE92CE9CD000915B
:100340006400013009F001C02DC00091640002304A
:1003500009F001C04AC0009160000B3009F00FC0E5
:1003600040D184E690E0CBD1ECE9F7E032D1A4E6CD
:100370008C918F5F8C9380E080936300B0CE00916E
:1003800060000C3009F00DC0EAE0F0E0A4E1EAD131
:10039000A1E60D911C910417150709F001C085C055
:1003A0005DC036C0009160000C3009F01DC0EAE06D
:1003B000F0E0A4E1D7D1A1E60D911C910417150737
:1003C00009F401C04BC0A1E6ADD180E08093630089
:1003D00080E080936500A4E68C918F5F8C9301D1BF
:1003E000E6EAF7E0F6D07BCE13C0009160000C3057
:1003F00009F00EC0EAE0F0E0A1E67BE7A2D1F1D07F
:10040000E0EBF7E0E6D040D0E2E0F0E0FBD04ACE0F
:10041000A3E68C918F5F8C930091630045E0040FFD
:10042000A5E60C938FEBA5E61C91EAD0E0ECF7E093
:10043000D0D0A1E60D911C914AE050E0B7D0A1E6E2
:100440000D931C93A1E60D911C91A0E64D915527AB
:10045000040F151FA1E60D931C930895C2D0E2EC82
:10046000F7E0B7D0939AE3E0F0E0CCD09398E4E1E2
:10047000F0E0C8D017CE939A84E690E040D19398EC
:1004800084E690E03CD1089584E690E038D1939AD8
:1004900088EC90E034D1939888EC90E030D1939A36
:1004A00088EC90E02CD1939808958091660081505B
:1004B00080936600E9E0F0E0A6E691E07BE742D1B8
:1004C00090D0E0EDF7E085D0DFDF909A81E090E01A
:1004D00016D1C89B01C0FACF9098D6DF82D081E0B8
:1004E0008093640000916400003110F009F00DC0A9
:1004F000E1E0F0E087D0E0ECF7E06BD0BCDFA4E611
:100500008C918F5F8C9308F4EDCF6BD0EAEDF7E020
:1005100060D0BADF919A81E090E0F1D082990BC06F
:1005200091985DD0E6EEF7E054D0939AE2E0F0E0E7
:1005300069D09398BACFC99B01C0EDCF9198A4DF41
:10054000B1CD4FD0B79901C00FC0EAE0F0E002EDA5
:1005500014E0A0E1BB277BE7F4D096DFE2EFF7E001
:1005600038D0E3E0F0E04ED0089504D01FD000FC76
:100570000CD008950024E89457FF02C009D0689475
:1005800000F80BD010F80124089502D009D0089586
:10059000509540954F5F5F4F0895E89417FF089579
:1005A000009510950F5F1F4F68940895752F642F65
:1005B00055274427FF93F1E1889405C010F4460FB6
:1005C000571F5695479517950795FA95B9F7FF91D7
:1005D0000895A4D0802D11F060D0FBCF089580EC59
:1005E00062C081E060D014D080E85DC08FE7213028
:1005F00039F08FEB223021F08FE8233009F08FECB7
:10060000810F51C088EE93E07AD03197D9F70895E1
:1006100083E0992774C08AEF90E071D0BB9ABA9AB0
:10062000B99AB89A8E9A8D9A959885E090E067D09D
:100630009698C398C298C19AC09A969AEF93FF93DE
:10064000E5E1F0E050D0FF91EF91969855D0969A61
:10065000EF93FF93E5E1F0E046D0FF91EF9196989C
:100660004BD0969AEF93FF93E5E1F0E03CD0FF91F9
:10067000EF91969841D0C098969AEF93FF93E5E159
:10068000F0E031D0FF91EF91969836D088E20BD010
:100690008EE009D086E007D00895959A829505D01E
:1006A00004D02AD008959598F9CF859510F4C09A72
:1006B00001C0C098859510F4C19A01C0C198859574
:1006C00010F4C29A01C0C298859510F4C39A01C073
:1006D000C398969AEF93FF93E5E1F0E004D0FF9181
:1006E000EF91969808953197F1F70895689462F81C
:1006F0000895E89462F8089581E090E000C0EF93D7
:10070000FF93EE27E82BE92B31F0EAEFF0E0319789
:10071000F1F70197D1F7FF91EF910895C8953196C0
:100720000020089582E001C084E099279D938A9576
:10073000E9F70895E199FECFEEBB3196089591E077
:1007400001C092E07B3751F47FB7F894F3DF8D91CD
:100750008DBBE29AE19A9A95C9F77FBF77270895F2
:1007600091E001C092E0E6DFE09A8DB38D939A9517
:10077000D1F708955757572E4156522E344D472ED4
:10078000434F4D00436F64654C6F636B0000202046
:1007900020456E74657220636F646500204F6C6441
:1007A00020636F646500204E657720636F64650089
:1007B00020436F6465206163636570746564000045
:1007C0002A00202020436F64652077726F6E6700D7
:1007D00020202020204F70656E0020202020204304
:1007E0006C6F736500002020202042617272696581
:1007F0007200436F64652069732031323334000026
:00000001FF
